:1000000012C0189518951895189518951895189563
:100010001895189518951895189518951895189578
:100020001895189518958FED8DBFC0ECE0EC4E2E0D
:10003000DD275D2EEEE7F0E0A0E6B0E088278D93A7
:100040003197E9F7D1D266248FE087BB8FEF81BB70
:1000500080E082BB8FE788BB80E08093630084E60A
:1000600090E036D38DE008D3BF98A8E69C9197FF27
:1000700004C0B7990EC09F779C93B79B0AC088E2D3
:100080009F93992725D39F91B79B03C090689C931A
:1000900029D290D2E6E4F7E085D2E2E0F0E09BD20C
:1000A00089D286D2E6E5F7E07DD284EF91E010D3E5
:1000B000ECE5F7E077D284EF91E00AD3E2E6F7E0EF
:1000C00071D284EF91E004D3E8E6F7E06BD2E1E08F
:1000D000F0E081D28CE0D0D280E080936600A1E68F
:1000E0000AD380E08093640080E08093670062D24E
:1000F000ECE6F7E057D288EC90E0EAD2E2E7F7E0EE
:1001000051D288EC90E0E4D2E4E7F7E04BD288ECFF
:1001100090E0DED2E6E7F7E045D288EC90E0D8D276
:10012000E8E7F7E03FD288EC90E0D2D2EAE7F7E0E8
:1001300039D288EC90E0CCD2EEE7F7E033D288EC0D
:1001400090E0C6D2E0E8F7E02DD288EC90E0C0D293
:10015000E6E7F7E027D2C39AC0988CE0809360006E
:10016000BC98A8E69C9196FF04C0B49B0EC09F7BF0
:100170009C93B4990AC088E29F939927A9D29F9132
:10018000B49903C090649C9381D080E08093600018
:10019000BD98A8E69C9195FF04C0B59B0EC09F7DBD
:1001A0009C93B5990AC088E29F93992791D29F9119
:1001B000B59903C090629C9369D08BE080936000F6
:1001C000BE98A8E69C9194FF04C0B69B0EC09F7E8B
:1001D0009C93B6990AC088E29F93992779D29F9100
:1001E000B69903C090619C9351D0C09AC19AC29AAB
:1001F000C39883E080936000BC98A8E69C9196FF2A
:1002000004C0B49B0EC09F7B9C93B4990AC088E243
:100210009F9399275DD29F91B49903C090649C935A
:1002200035D082E080936000BD98A8E69C9195FF50
:1002300004C0B59B0EC09F7D9C93B5990AC088E20F
:100240009F93992745D29F91B59903C090629C9343
:100250001DD081E080936000BE98A8E69C9194FF39
:1002600004C0B69B0EC09F7E9C93B6990AC088E2DC
:100270009F9399272DD29F91B69903C090619C932B
:1002800005D08AE090E024D266CFE9CE939A84E646
:1002900090E01ED2939884E690E01AD20091660016
:1002A000013009F001C05AC000916600023009F027
:1002B00001C07BC0009160000B3009F00FC0B699FF
:1002C00001C0FDCF77D1E2E8F7E06CD1A6E68C91D2
:1002D0008F5F8C9380E080936400089500916000AC
:1002E0000C3009F00DC0EAE0F0E0A4E124D2A1E670
:1002F0000D911C910417150709F001C0D6C069C003
:10030000A4E68C918F5F8C930091640044E0040F0D
:10031000A7E60C938FEBA7E61C915BD1E2E9F7E02F
:1003200041D100916400083010F009F001C001C013
:1003300050C0A1E60D911C914AE050E020D1A1E609
:100340000D931C93A1E60D911C91A0E64D915527AC
:10035000040F151FA1E60D931C93089500916000F2
:100360000C3009F021C0EAE0F0E0A4E1E4D1A1E61C
:100370000D911C910417150709F401C02AC0A1E6CC
:10038000BAD180E08093640080E080936700A6E6A5
:100390008C918F5F8C930ED10DD188EC90E098D129
:1003A000E4E9F7E0FFD00895ABCF009160000C3096
:1003B00009F00EC0EAE0F0E0A1E67BE7ABD1FAD0AD
:1003C000E4EAF7E0EFD060D0E2E0F0E004D184CEE0
:1003D00097CF939AEFD0E4EBF7E0E4D084EF91E08D
:1003E00077D1E8D084EF91E073D1E4EBF7E0DAD095
:1003F00084EF91E06DD1DED084EF91E069D1E4EB40
:10040000F7E0D0D09398E1E0F0E0E5D0D1D0E2EC95
:10041000F7E0C8D0E1E0F0E0DED0E2E9F7E0C2D0FA
:10042000E1E0F0E0D8D0E2E9F7E0BCD0E1E0F0E0D4
:10043000D2D0E2E9F7E0B6D0E1E0F0E0CCD0E2E9FA
:10044000F7E0B0D0E1E0F0E0C6D0E2E9F7E0AAD012
:10045000E1E0F0E0C0D0E2E9F7E0A4D0E1E0F0E0D4
:10046000BAD0E2E9F7E09ED0E1E0F0E0B4D0E2E912
:10047000F7E098D0E1E0F0E0AED0E2E9F7E092D02A
:10048000E1E0F0E0A8D028CE84E690E021D1939A74
:1004900088EC90E01DD1939888EC90E019D1939A64
:1004A00088EC90E015D193980895A3E68C918F5F26
:1004B0008C9384E190E00CD17DD0E4EAF7E072D037
:1004C000E3DF76D0E8ECF7E06DD08CE291E000D18C
:1004D000949AE2E0F0E07FD094986CD0E1E0F0E014
:1004E0007AD0DECD67D0B79901C025C0EAE0F0E050
:1004F0000EEC14E0A0E1BB277BE70CD1C5DF8FE059
:10050000BBD058D0E6EDF7E04DD084EF91E0E0D0DD
:10051000E0EEF7E047D084EF91E0DAD049D0E6EEA4
:10052000F7E040D084EF91E0D3D0EEEEF7E03AD0A0
:10053000E2E0F0E050D08CE09FD0089504D01FD0CE
:1005400000FC0CD008950024E89457FF02C009D0A5
:10055000689400F80BD010F80124089502D009D057
:100560000895509540954F5F5F4F0895E89417FFA9
:100570000895009510950F5F1F4F68940895752F8B
:10058000642F55274427FF93F1E1889405C010F4A8
:10059000460F571F5695479517950795FA95B9F742
:1005A000FF910895A4D0802D11F060D0FBCF089565
:1005B00080EC62C081E060D014D080E85DC08FE73D
:1005C000213039F08FEB223021F08FE8233009F011
:1005D0008FEC810F51C088EE93E07AD03197D9F734
:1005E000089583E0992774C08AEF90E071D0BB9A98
:1005F000BA9AB99AB89A8E9A8D9A959885E090E0B1
:1006000067D09698C398C298C19AC09A969AEF9369
:10061000FF93E5E1F0E050D0FF91EF91969855D02F
:10062000969AEF93FF93E5E1F0E046D0FF91EF91CA
:1006300096984BD0969AEF93FF93E5E1F0E03CD08B
:10064000FF91EF91969841D0C098969AEF93FF93BF
:10065000E5E1F0E031D0FF91EF91969836D088E255
:100660000BD08EE009D086E007D00895959A829548
:1006700005D004D02AD008959598F9CF859510F427
:10068000C09A01C0C098859510F4C19A01C0C19864
:10069000859510F4C29A01C0C298859510F4C39A4A
:1006A00001C0C398969AEF93FF93E5E1F0E004D080
:1006B000FF91EF91969808953197F1F70895689416
:1006C00062F80895E89462F8089581E090E000C02F
:1006D000EF93FF93EE27E82BE92B31F0EAEFF0E000
:1006E0003197F1F70197D1F7FF91EF910895C895F0
:1006F00031960020089582E001C084E099279D93FF
:100700008A95E9F70895E199FECFEEBB31960895F9
:1007100091E001C092E07B3751F47FB7F894F3DFAA
:100720008D918DBBE29AE19A9A95C9F77FBF7727A1
:10073000089591E001C092E0E6DFE09A8DB38D93D9
:100740009A95D1F708955757572E4156522E344D4A
:10075000472E434F4D00436F646500004C6F636B41
:100760000000204156520000204C5400202020451B
:1007700000006E00740065007200206300006F00CE
:10078000640020456E746572206F6C6420636F6432
:1007900065002A0020456E746572206E65772063BF
:1007A0006F64650020436F646520616363657074E6
:1007B00065640000202020436F64652077726F6EAF
:1007C00067002020202A000020202020556E6C6F1A
:1007D000636B656400002020496E697469616C0078
:1007E00020636F6465002020202020697300202092
:0607F0002031323330001D
:00000001FF
